:020000040000FA
:1000000000008A1118280034F200030E8301F10069
:100010000A088A01F000040883120313B100840067
:1000200070088A008301710E8300F20E720E0900BF
:100030004530FE000130FF0080308A11000024218D
:100040008A11000083120313A1007F08A00047302B
:10005000A2000130A300831203132008A40021088A
:10006000A500FF30A007031CA103240825040319E1
:10007000A82804302207A400A501A50D2308A50780
:100080002408FE002508FF0080308A11000024218A
:100090008A11000083120313A7007F08A60022081C
:1000A000FE002308FF0080308A11000024218A11FD
:1000B000000083120313A900A5007F08A800A40074
:1000C00002302207A400A501A50D2308A5072408D6
:1000D000FE002508FF0080308A11000024218A11CB
:1000E000000083120313A500AB007F08A400AA0040
:1000F000831203132608AA002708AB00FF30A607C7
:10010000031CA7032A082B040319A1282808FE00B2
:100110002908FF0080308A11000011218A11000097
:1001200083120313AA00240884008313251883175D
:100130002A088000A80A0319A90AA40A0319A50A13
:100140007828063083120313A2070318A30A2B286A
:100150008A110000AC280800023083120313AC009F
:10016000831203179E019F01FF308316031385003E
:10017000FF308600FF308700071087108711831239
:100180000313AD01AE018312031306088312031398
:10019000AF002C08013A031DD028AD0A0319AE0A9E
:1001A0002730831203132E02031DD82811302D028D
:1001B000031CE028023083120313AC00AD01AE0132
:1001C000103083120313AF052F08031DE9280130F7
:1001D000AC00831203132C08013A031DF328831289
:1001E000031387140710831203132C08023A031D0C
:1001F000FD288312031307148710831203132F089B
:10020000003003190130B000300C03180A298312A2
:1002100003138711031C0F29831203138715C328A7
:100220000800003A03191829803A03191F290034DD
:100230007E08840083137F188317000808007F0856
:100240008A007E0882000800003A03192C29803AAF
:1002500003193629FF0100347E08840083137F18B8
:1002600083170008FF00840A000808008A110000B4
:100270001F21FD00FE0FFF03FF0A8A1100001F214E
:10028000FC007D08FF007C080800013400340334C2
:0A029000003432340034013400342D
:02400E00D430AC
:00000001FF
